:020000040000FA
:02000000092ACB
:08000800A000030E8312A10009
:100010002608820020342034203420342034203438
:100020006534733463342E34613473346D34203466
:10003000563431342E3435342034203420342034B6
:100040004534533443344334203420342034203472
:10005000B801B901BA01B90AB601B7010310B50D6B
:10006000B80D03183628B90DBA0D2E28B80CB50CEA
:100070003508B3023808031C013EB402031C4C28A7
:100080003908B6043A08B7040310BA0CB90C0318BF
:100090000800B80CB50C38283508B3070318B40AA3
:1000A0003808B4074428B601B7013508B800381C31
:1000B0005F283308B60734080318013EB70703105A
:1000C000B80C3808031908000310B30DB40D5728F5
:0C00D000313E8200713E8200B13E820091
:1002000085010000062A27088500082200008501D4
:10021000062A2708850005292708850000000B29E4
:10022000270885000E2927088500000012292708C5
:100230008500152927088500000019292708850051
:1002400000001C2927088500042A000085010822D7
:10025000292927088500042A000085010822302961
:100260002729003400340034033409340C341034AA
:10027000133417341A341E34F134F134F134F134B8
:10028000F134F134F134F134F134F134F134F13446
:10029000F134F134F134F134F134F134F134F13436
:1002A000F134F134F134F134F134F134F134F13426
:1002B000F134F134F134F134F134F134F134F13416
:1002C000F134F134F134F134F134F134F134F13406
:1002D000F134F134F134F134F134F1342C34253487
:1002E000223400340034003400340034003400344C
:1002F0000034003400340034FB34FA34F834F7347A
:10030000F534F334F134EF34ED34EB34E934E734DD
:10031000E434E234DF34DC34D934D634D234CF346C
:10032000CB34C734C334BE34B934B434AE34A83457
:10033000A1349A34923489347F34753469345C340E
:100340004D343C3429341334093409340934093424
:1003500009340934093409340934093408340834B7
:100360000834083408340834C834C834C834C834AD
:10037000C834C834C834C834C934C934C934C93499
:10038000C934C934C934C934C934C934C934C93485
:10039000C934C934C934C934C934C934C934C93475
:1003A000C934C934C934C934C934C934C934C93465
:1003B000C934C934C934C934C934C934C934C93455
:1003C000C934C934C934C934CD34D334D934DE3412
:1003D000E434E934EE34F334F834FC3400340034DB
:1003E0000034A218F829A214000085012908FD296B
:1003F000270885002808A210000081000B11210E9B
:100400008300A00E200E09002808FD292908FD29D7
:1004100008008316FF239000831201308A008501B3
:100420008316303001389F00103095000030810075
:10043000DF30FB3985008312FF3081008B160130DD
:100440009F00A2011430A300A501A701A801A901E2
:10045000F130A600FF30AF00B000B100B2008B1742
:10046000F0222218302A4308BC00BE004208BB001C
:10047000403EBD000318BE0AF02222183C2A420862
:100480003D024308031C013E3E0203183C2A420879
:10049000BD004308BE003B083D02B300AD003C0870
:1004A000031C013E3E02B400AE004030B5002820DF
:1004B0003608AC00B300B40153203608AD0237084B
:1004C000031C013EAE020310AE0CAD0C3B08AD07A1
:1004D0003C080318013EAE07F02222186C2A3D08A2
:1004E00042023E08031C013E43020318472A420809
:1004F000B3004308B4001B230038031D6C2A8B177C
:10050000D622E322D6228B17A501A701C6222308F3
:10051000A40014232218872A6820003C031D872A80
:10052000A40B892A0130A300A7018501A501C622D9
:100530002030A70014232218842A25020319AC2A8C
:100540000318A62AA50AC62222119A2A221DAA2A1F
:10055000A502C62222159A2A22112608003C031D54
:100560009A2A851D9A2A0430A7000130A500C622C8
:1005700014232218842A6820003C031D942A250A8B
:100580003F3C031CB82AA50AC622B82A25086A20BF
:10059000AA0025086C20AB00250868208B12A60055
:1005A0002A08A8002B08A9008B160800C830BF0035
:1005B0002030850008220822082208228501E9222D
:1005C000BF0BD82A0800C830BF00E922BF0BE52ABC
:1005D000080064003230C0000822C00BEC2A08007A
:1005E0002F23221808000530C1000E08C2000F0892
:1005F000C3002F23221808004208FD3EB300430821
:10060000031CFF3EB40033080E02B3003408031C81
:10061000013E0F02B400031DF02A07303302031815
:10062000F02AC10BF92A08002F23221800340E08E3
:10063000B3000F08B4002D08B3022E08031C013EBE
:10064000B402031C00342C08B5002820B708031D91
:100650003F344030360203183F3436080800221079
:100660004030C4001B30C5008E018F014130900026
:100670005C23221800340E080F040319382B0330B2
:100680009F005C232218003409300F020318562BF8
:10069000051E412B90019F18612B6323553C0318C5
:1006A000612B03300F02031C342B08005C2322183B
:1006B0000034051E562B342B6400C40B0800C50BF8
:1006C0000800221408003108B2003008B1002F08D9
:1006D000B0001E08AF00C600C7013008C6070318E7
:1006E000C70A3108C6070318C70A3208C607031825
:0E06F000C70AC70CC60CC70CC60C460808008B
:02400E00CC3FA5
:00000001FF
